:100000000010001015010000D5000000D90000000C
:1000100000000000000000000000000000000000E0
:10002000000000000000000000000000DD000000F3
:100030000000000000000000E10000005D0600007C
:10004000E5000000E500000000000000E500000001
:10005000E5000000E500000000000000E5000000F1
:10006000E5000000E5000000E5000000E5000000FC
:10007000E5000000E5000000E5000000E5000000EC
:10008000E5000000E5000000E5000000E5000000DC
:10009000E5000000E5000000E500000000000000B1
:1000A000E5000000E5000000E5000000E5000000BC
:1000B000E5000000E5000000E5000000E5000000AC
:1000C000EC110000000000101000000010000010F3
:1000D000E4010000FEE7C046FEE7C046FEE7C0467A
:1000E000FEE7C046FEE7C04610B5002304E0046802
:1000F0000C600433043004319342F8D310BDC04681
:10010000002303E000220260043304308B42F9D361
:100110007047C04610B50D4B07E0186859681C1CA5
:100120000C349A68FFF7E0FF231C094A9342F4D38A
:1001300006E018681C1C08345968FFF7E1FF231C0F
:10014000044A9342F5D300F055FCFEE7C0000000DE
:10015000CC000000D400000090B583B000AF041CB8
:10016000081C111CFB1D221C1A70BB1D021C1A70DE
:100170007B1D0A1C1A70094BFA1D12781A70074B66
:10018000BA1D12785A70054B7A1D12789A700120A8
:1001900000F02EF8BD4603B090BDC0461000001020
:1001A000B0B582B000AF051C0C1C101C191CBB1D87
:1001B0002A1C1A803B1D221C1A80BB1C021C1A80A0
:1001C0003B1C0A1C1A80094BBA1D12889A80074BE7
:1001D0003A1D12881A81054BBA1C1288DA80034B2B
:1001E0003A1C12885A81BD4602B0B0BD1000001002
:1001F00080B582B000AF021CFB1D1A70FB1D1A787F
:10020000062A4BD81B789A002C4BD3181B689F46A4
:100210002B4BFA2252009A80294BFA2252001A8163
:10022000274BFA225200DA80254BFA2252005A81DB
:1002300041E0234BFA229A80214BFA221A81204B6B
:10024000FA22DA801E4BFA225A8134E01C4B6422D7
:100250009A801B4B64221A81194B6422DA80184B56
:1002600064225A8127E0164B32229A80144B3222A4
:100270001A81134B3222DA80114B32225A811AE052
:100280000F4B64229A800E4BC8221A810C4B6422B9
:10029000DA800B4B962292005A810CE0084B3222F6
:1002A0009A80074B64221A81054B3222DA80044B74
:1002B000962252005A81BD4602B080BD94110000C2
:1002C0001000001080B500AF002000F041F8BD46DE
:1002D00080BDC04680B582B000AF021CFB1D1A7005
:1002E000FB1D1B78002B15D0164B9B78002B08D0DC
:1002F000144B5B781A1C012393401A1C124B1A6092
:100300001DE0104B5B781A1C012393401A1C0F4B05
:100310001A6014E00B4B9B78002B08D0094B5B78DC
:100320001A1C012393401A1C084B1A6007E0054B66
:100330005B781A1C012393401A1C034B1A60BD46BC
:1003400002B080BD10000010002200A0802200A09A
:10035000B0B584B002AF78607B68002B5CD07B685E
:100360001B78022B1CD002D8012B05D071E0032B87
:100370002AD0042B3CD06CE00120FFF7ABFF374BB9
:100380001C78374B9B88181C00F0FCFA051C0223D4
:100390000093201C022100222B1C00F0FFFA58E0E1
:1003A0000020FFF797FF2D4B1C782D4B1B89181C45
:1003B00000F0E8FA051C02230093201C0321002210
:1003C0002B1C00F0EBFA44E00120FFF783FF234BE6
:1003D0001C78234BDB88181C00F0D4FA051C022380
:1003E0000093201C042100222B1C00F0D7FA30E0DF
:1003F0000020FFF76FFF194B1C78194B5B89181C05
:1004000000F0C0FA051C02230093201C01210022E9
:100410002B1C00F0C3FA1CE0124B1B68104A5278E8
:10042000111C01228A401A430E4B1A600E4A0F4BD0
:10043000101C191C00F0BCF9031C191C074B0A1CEA
:100440001A7002230093081C01210022002300F0EF
:10045000A5FA0023181CBD4602B0B0BD0000001074
:1004600010000010002000A051030000B011000097
:1004700080B500AF0D490E4A0E4B042000F0F6F88F
:1004800000F01AF800200C210022FFF765FEC823B7
:100490005B000A2050210A22FFF782FEFFF712FFBD
:1004A000002000F057F8BD4680BDC046001BB700D5
:1004B0000087930380C3C90180B500AF244B1B683C
:1004C00001221A43224B1A60214B1B6802221A4355
:1004D0001F4B1A601E4B1B6810221A431C4B1A60DC
:1004E0001B4B1B6840221A43194B1A60184B1B68A0
:1004F00080221A43164B1A60154B1B68802252004B
:100500001A43134B1A60124B1B68802292001A4345
:100510000F4B1A600E4B1B688022D2001A430C4B03
:100520001A600B4B1B68802212011A43084B1A6099
:10053000074B1B68802252011A43054B1A60044B7B
:100540001B68802292011A43014B1A60BD4680BD90
:10055000002000A090B585B002AF78607B68002BCA
:1005600055D07B681B78002B66D1364B1B78002B4F
:1005700026D0344B00221A70334B01221A60324BC2
:1005800002221A60304B10221A602F4B40221A6050
:100590002D4B80221A602C4B802252001A602A4B6D
:1005A000802292001A60284B8022D2001A60264BCB
:1005B000802212011A60244B802292011A603BE0D3
:1005C000204B01221A70214B01221A601F4B02227C
:1005D0001A601E4B10221A601C4B40221A601B4BE3
:1005E00080221A60194B802252001A60174B802219
:1005F00092001A60154B8022D2001A60134B8022A1
:1006000012011A60114B802292011A6014E0104A04
:10061000104B101C191C00F0CBF8031C191C0E4BBE
:100620000A1C1A7032235C4202230093081C00212A
:100630000022231C00F0B2F90023181CBD4603B0B1
:1006400090BDC0461C000010002200A0802200A027
:1006500055050000C011000001000010024A136897
:10066000013313607047C04620000010032802D0F9
:10067000042838D077E03D490A603D4A13603D4B7D
:100680008E2189005A58022082435A500021196451
:1006900001225A6459645A64364B5B6CDB07FBD504
:1006A000344B40229A608E2189005A588020824320
:1006B0005A50304BDB68DB07FBD52E4B03221A6701
:1006C000023A5A67002159675A672A4B5B6FDB076A
:1006D000FBD5284B02229A6727497E329950012187
:1006E000143299503FE021490A60214A1360214B9E
:1006F0008E2189005A58202082435A5000221A62C3
:10070000002301E0C0460133C72BFBD9194B002160
:10071000196401225A6459645A64164B5B6CDB07F6
:10072000FBD5144B24229A608E2189005A588020D0
:1007300082435A500F4BDB68DB07FBD50D4B03227E
:100740001A67023A5A67002159675A67094B5B6F6B
:10075000DB07FBD5074B02229A6707497E32995087
:1007600001211432995000207047C0460400001047
:100770000800001000800440DF000500014B1868ED
:100780007047C04608000010014B18687047C0460B
:1007900020000010002305E099000020034A885043
:1007A0000133DBB21E2BF7D9002070472400001064
:1007B000F0B583B0002827D0002401E00134E4B272
:1007C000251CA300124A9B58002B01D01D2CF5D9E3
:1007D0001D2C14D80191071C2C2000F019F9061EBD
:1007E0000FD000212C2200F00EF93760019B7360BE
:1007F0000023B361F361AD00054BEE5002E0F52438
:1008000000E0FA24201C00E0FC2003B0F0BDC0464C
:100810002400001010B51D281ED880000F4C005970
:10082000047C002C0DD02923C35C622B04D8013337
:1008300029228354F52010E063222923C254F52095
:100840000BE00172C2602822835443690133436183
:1008500001230374002000E0FC2010BD24000010E0
:10086000F8B5FFF791FF314B1D68A84201D3451B36
:1008700000E0451B2D4B186000241BE09A69002AFC
:1008800016D0AA4202D9521B9A6111E000229A6145
:10089000274E8F00BB592032995C5A6A28201B5C76
:1008A000201CFFF7B7FFBB59DA69002A00D09A6114
:1008B0000134E4B2211CA3001D4A9B58002BDDD15A
:1008C00001261E25002420E0037C002B1BD02822BB
:1008D000825C012A02D0022A08D014E000230374AB
:1008E0000368002B0FD0083098470CE00133DBB2CF
:1008F0000374142B03D89BB2B34202D803E0251C27
:1009000001E01E1C251C0134E4B2A300084A9858DB
:100910000028D9D11D2DA4D8131CAD000022E95800
:100920000A74E8580368083098479AE7A000001056
:100930002400001008B5FFF72DFFFFF799FDFFF722
:100940001DFFFA21890000F0A6FB01380A4B9842EE
:1009500010D80002000A0138084A506008490B6AA2
:100960001B021B0AC020000603430B620023936096
:1009700007331360FFF774FFFFFFFF0010E000E094
:1009800000ED00E008B5FA239B005843024B1968BC
:1009900000F081FB08BDC0460C00001070B504AC2F
:1009A0002578FF2820D08400114EA459002C1DD09A
:1009B000002B03D12B1CFFF72DFF18E0002B09DDC6
:1009C0002020215462622822A5540022E261A36102
:1009D00000200CE02020215462622822A5545B42B2
:1009E000E361A361002002E0FF2000E0FF2070BD72
:1009F00024000010002008B5011C021C00F096F82D
:100A0000FFF798FF08BD08B500F07FFB08BD0000A8
:100A1000F7B5314EC51C3468AD080196002813D0D7
:100A20008022291CEB1C002752050A319C4604E059
:100A30002368934213D0271CA468002CF8D10C30F3
:100A400000F0ECF8431C0FD1002043E03E689642D2
:100A500017D17E689B1903336360BB68A360A768E6
:100A60006368002FF2D10CE080239B050360456092
:100A70008460002F02D1019B186000E0B8600C3048
:100A800028E0AB4205DB9C4503DB80239B0523600C
:100A90001EE08B4210D98022201C8021920522600A
:100AA0000C30AA005B1B82184905033B6560A260FD
:100AB0001160536097600DE0002FBCD19B00C01AFD
:100AC00000F0ACF8431CBFD080239B052360656019
:100AD000201CD4E7FEBDC046A800001010B50028B9
:100AE00012D080235B05191C0C3803608268002A31
:100AF0000AD013688B4207D1546843681B1903332B
:100B0000436093688360F1E710BD000010B5FFF704
:100B10007FFF041E05D10449172200F035FB00F0C9
:100B200009FB201C10BDC046CD110000A02238B525
:100B3000224C00215200201CFFF765FFC020FFF768
:100B4000E5FF1F4D0021C0222860FFF75CFF002356
:100B50002868282218215A435943A2184118013302
:100B60005162082BF5D1221C1649002000F098F89C
:100B700080228023201C5B010021D20000F02AF893
:100B8000114D124C291C221C012000F089F88022F2
:100B90008023201C5B010021D20000F01BF80C4CCC
:100BA000291C221C022000F07BF880228023201CBC
:100BB0000021D2005B0100F00DF838BDB400001038
:100BC000B0000010E5110000E7110000DC0000108B
:100BD00004010010F0B5C5680124AE071AD08026C4
:100BE000B600B2420BD08026F600B24204D0802676
:100BF0007600B2420ED102E0416A231C04E0064EA8
:100C00005F1E0124B74205D800241543016101602D
:100C1000C361C560201CF0BDFEFFFF0070B50C4D28
:100C20002B68002B01D10B4B2B600323C41C2E68B7
:100C30009C433419201C00F0FBF9002802D12C60E1
:100C4000301C04E00C220120034B40421A6070BDAE
:100C5000AC000010F4010010A4000010202310B517
:100C6000041CC2689A43436AE2605B6882699A42E4
:100C70000DD000F049F8E268074B134010221343EF
:100C8000626AE3605368A361236993602360E2684A
:100C9000024B1340E36010BDEFCFFFFFBFBFFFFF6C
:100CA00070B50D1C061C101C141C00F095F82B7858
:100CB000722B09D0772B04D0612B20D10823114A45
:100CC00004E00423022201E00023012201352978F7
:100CD0002B2905D0622908D104210A43033902E0F7
:100CE00003210A4301390B43F0E7E26066611B0709
:100CF00006D5201C0021022200F0C0F800E00024EC
:100D0000201C70BD0280000038B5436AC268996833
:100D1000144B05691340C360822304681340022BFF
:100D200002D001235B421BE080235B02134017D0FB
:100D3000A14200D2211C041CA94209D1636AE168C6
:100D40009D600023084A25600A40A360E26007E036
:100D5000491B281C221C00F009F80028EED0E0E70F
:100D6000181C38BDFFFFF7FFFFFFFEFFF7B5D66881
:100D700001900D1C141C5769F30205D51023381C73
:100D80001E4300F0E3F9A061114B1E4209D0381C4C
:100D9000A16900F0EDF98023002811DB0D4B1E4006
:100DA000E6602A1C381C019900F0EEF943005B084C
:100DB000ED1AA3695D190023A561984205D080331F
:100DC000E2681343E36001235B42181CFEBDC0468A
:100DD00010000200EFFFFDFFF0B5436AC5688BB05D
:100DE000476906690193AB0727D0041C2B0716D46B
:100DF00000F02AF8381C00F0A3F92B0502D5301CAE
:100E0000FFF76CFE0F4BAD0DAD059D4207D102A85B
:100E1000216A202200F0B2F902A800F0D5F80021E2
:100E20001822606AFFF7EFFD201C00212822FFF73F
:100E3000EAFD019B0020636201E0012040420BB00B
:100E4000F0BDC046000080AD38B5002803D000F0EA
:100E5000F9F8051C0EE0041C051C0748201800F0DA
:100E6000F1F8002801D001256D42A02328345B0051
:100E70009C42F2D1281C38BDB4000010F7B5C368FD
:100E8000161C0093009A3B4B041C0D1C47691A4228
:100E90006BD0381C00F060F90190002865D1012E5C
:100EA00004D0022E07D0002E5FD124E0201C00F0D9
:100EB00065F82D181FE0381C00F048F9002805DA05
:100EC0008023E2681343E36001234FE0626A2168F4
:100ED0009368994200D90B1CA1695B1821695B1AC0
:100EE000E168890603D55268934200DA131C8342F5
:100EF00000DA031CED18002D37DB009B616A9B04B0
:100F000004D523688A689A4200D28B60A3699D4207
:100F10000DDB20688A68824200D2021C2069D61844
:100F2000361AB54203DCCF68DE19B54207DB202351
:100F3000009A13430022A26062604D6011E0ED1A36
:100F4000009B9B0701D5EF1BA760009BDB0702D529
:100F5000821AAA1862602023009A45199A43131C2A
:100F60002560054A1340E36001E0022301930198E4
:100F7000FEBDC04603001000BFCFF7FFC3689A074D
:100F800005D1212201200F4B40421A6018E0202297
:100F900019030BD5134202D0436A586804E0036872
:100FA000826900699B18181A013809E0134202D0BF
:100FB000436A586804E00368826900699B18181A3C
:100FC0007047C046A400001010B5041C00F006F8DD
:100FD000011C201C00F0C6F810BD000010B5431C19
:100FE000820706D00130421E1278002AF8D1C01ABA
:100FF00018E002680C490D4C51189143214201D16F
:101000000430F6E7D4B2411C002C0AD0FF2424029D
:10101000811C224205D0FF242404C11C224200D09E
:10102000011DC81A10BDC046FFFEFEFE80808080F4
:10103000034B021C181E02D000209A424041704708
:10104000000000000323C26870B51340041C181E82
:101050001AD0930605D5636A201C5E68FFF7FEFD73
:1010600004E02368A2699E182369F61AE268074B18
:10107000201C1340E360FFF747FE051C311C201CB9
:101080000022FFF7FBFE281C70BDC046FFCFFFFF0C
:1010900003000B4321D4002931D00122D2070309D8
:1010A00001E0090112099942FBD9430801E0490016
:1010B00052089942FBD900E04908401A07D352412F
:1010C000FAD301461046704749084018F7D29218E3
:1010D000FAD34018014610467047CB0F00D0494262
:1010E000021000D54042534008B5FFF7D4FF0CBCB6
:1010F000521000D34042002A00D549421847F44616
:10110000002000F001F8604770478446043A09D394
:10111000830707D109060B0A19430B0C1943043A3C
:1011200002C0FCD2043203D001700130013AFBD17D
:101130006046704718200149ABBE70472600020088
:1011400003B469460220ABBE02B0704703B46946DF
:101150000C20ABBE02B0704703B469460920ABBE99
:1011600002B0704703B469460E20ABBE02B07047B0
:1011700003B469460A20ABBE02B070470FB469469B
:101180000D20ABBE04B070470FB469460520ABBE5E
:1011900004B070479C0200009C0200008002000026
:1011A00010020000320200004C0200006602000043
:1011B00048454152547376635F74736B00000000BE
:1011C00063323134615F746F67676C65002A2A2A65
:1011D000205F437379735F616C6C6F632066616934
:0C11E0006C65640A0072007700FFFFFFDE
:1011EC00FFFF0000001BB700001BB700E803000066
:0400000300000115E3
:00000001FF
